:020000040800F2
:10000000580700208D040008610200086302000800
:10001000670200086B0200086F0200080000000081
:100020000000000000000000000000007302000853
:10003000750200080000000077020008790200083D
:10004000A7040008A7040008A7040008A7040008E4
:10005000A7040008A7040008A7040008A7040008D4
:10006000A7040008A7040008A7040008A7040008C4
:10007000A7040008A7040008A7040008A7040008B4
:10008000A7040008A7040008A7040008A7040008A4
:10009000A7040008A7040008A7040008A704000894
:1000A000A7040008A7040008A7040008A704000884
:1000B000A7040008A7040008A7040008A704000874
:1000C000A7040008A7040008A7040008A704000864
:1000D000A7040008B3140008A7040008A704000838
:1000E000A7040008A7040008A7040008A704000844
:1000F000A7040008A7040008A7040008A704000834
:10010000A7040008A7040008A7040008A704000823
:10011000A7040008A7040008A7040008A704000813
:10012000A7040008A7040008A7040008A704000803
:10013000A7040008A7040008A7040008A7040008F3
:10014000A7040008A7040008A7040008A7040008E3
:10015000A7040008A7040008A7040008A7040008D3
:10016000A7040008A7040008A7040008A7040008C3
:10017000A7040008A7040008A7040008A7040008B3
:10018000A7040008A704000800F002F800F041F8F6
:100190000AA090E8000C82448344AAF10107DA45E2
:1001A00001D100F036F8AFF2090EBAE80F0013F0F3
:1001B000010F18BFFB1A43F0010318470416000093
:1001C00024160000103A24BF78C878C1FAD8520724
:1001D00024BF30C830C144BF04680C6070470000C1
:1001E0000023002400250026103A28BF78C1FBD840
:1001F000520728BF30C148BF0B607047642901F027
:10020000DF81002070471FB501F0D4FA1FBD10B583
:1002100010BD01F09DFA1146FFF7F5FF00F008F858
:1002200001F0BBFA03B4FFF7F2FF03BC01F0E2F800
:1002300000244FF4E13001F0EAF8542001F058F8BE
:1002400008E0214604A001F07BF94FF4FA7001F0B8
:10025000B1F8641CF5E70000743A25640D0A00004B
:10026000704700BFFEE700BFFEE700BFFEE700BF2C
:10027000FEE7704770477047704700000CB50020DC
:10028000019000907648006840F48030744908601E
:1002900000BF7348006800F4003000900198401CD3
:1002A0000190009818B90198B0F5A04FF1D16C48B1
:1002B000006800F4003010B10120009001E000203F
:1002C00000900098012846D165484030006840F011
:1002D00080506349403108606248006840F4404003
:1002E000604908605E48083000685D490831086070
:1002F0000846006840F4004008600846006840F482
:10030000A05008605848091F0860081F006840F0A6
:100310008070091F086000BF5148006800F000703D
:100320000028F9D040F20570504908604C48083068
:10033000006820F003004A49083108600846006858
:1003400040F00200086000BF45480830006800F037
:100350000C000828F8D10CBD10B54548006840F4E1
:100360007000434908603E48006840F001003C4985
:10037000086000203A4908310860394800683D4962
:100380000840374908603C48091D0860081F00689C
:1003900020F48020091F0860002031490C310860DA
:1003A000FFF76CFF4FF0006031498039086010BDE5
:1003B00070B500200022022300240221284D0835B8
:1003C0002D6805F00C0020B1042806D0082834D18F
:1003D00007E02A4D2A4E356033E02A4D284E35601D
:1003E0002FE01F4D2D1D2D68C5F380541C4D2D1D74
:1003F0002D6805F03F0154B1224DB5FBF1F5184EC3
:10040000361D3668C6F3881605FB06F209E01B4D5B
:10041000B5FBF1F5124E361D3668C6F3881605FB9E
:1004200006F20F4D2D1D2D68C5F301456D1C6B00A7
:10043000B2FBF3F5124E356003E0104D104E3560FF
:1004400000BF00BF064D08352D68C5F303150E4EDD
:10045000705D0B4D2D68C540094E356070BD0000C4
:10046000003802400070004008544007003C024041
:1004700088ED00E0FFFFF6FE103000240024F400B9
:100480000000002000127A00040000200948804784
:1004900009480047FEE7FEE7FEE7FEE7FEE7FEE766
:1004A000FEE7FEE7FEE7FEE704480549054A064B7E
:1004B0007047000059030008890100085801002016
:1004C00058070020580300205803002032490143F8
:1004D000324A1160704770B5002100230F22C478A2
:1004E0001CB32E4C246804F4E064C4F5E064C4F347
:1004F0000721C1F10404E3B20A4144789C40E1B20F
:100500008478144021430C07210E254C0578615551
:10051000047804F01F050124AC4005786D11AD008E
:1005200005F1E025C5F8004109E0047804F01F0555
:100530000124AC401B4D0678761145F8264070BD6D
:10054000194A0A400243154B1B1F1A60704739B104
:10055000124A121D12680243104B1B1D1A6006E05E
:100560000E4A121D126882430C4B1B1D1A60704705
:10057000042808D14FF0E021096941F004014FF04F
:10058000E022116107E04FF0E021096921F0040148
:100590004FF0E022116170470000FA050CED00E019
:1005A00000E400E080E100E080FFFF1F10B504469A
:1005B0009848844208D10121084600F086FB0021BA
:1005C000012000F082FB76E09348844208D10121AB
:1005D000022000F07AFB0021022000F076FB6AE0A6
:1005E0008E48844208D10121042000F06EFB0021D6
:1005F000042000F06AFB5EE08948844208D10121B2
:10060000082000F062FB0021082000F05EFB52E0B1
:100610008448844208D10121102000F056FB0021BB
:10062000102000F052FB46E07F48844208D10121AF
:10063000202000F04AFB0021202000F046FB3AE099
:100640007A48844208D10121402000F03EFB00217D
:10065000402000F03AFB2EE07548844208D1012189
:10066000802000F032FB0021802000F02EFB22E0F1
:100670007048844208D10121801500F026FB00213A
:10068000A01500F022FB16E06B48844208D101213E
:10069000401500F01AFB0021601500F016FB0AE07F
:1006A0006648844207D10121001500F00EFB0021AD
:1006B000201500F00AFB10BDF0B50A46002100230A
:1006C000002400BF3DE0012505FA01F3156805EAA5
:1006D00003049C4234D105684F000326BE40B54355
:1006E000056015794E00B5400668354305601579FB
:1006F000012D02D01579022D16D185684F000326F1
:10070000BE40B543856055794E00B5408668354397
:100710008560456801268E40B543456045689679F9
:100720008E40B6B235434560C5684F000326BE40D3
:10073000B543C560D5794E00B540C6683543C56040
:10074000491C1029BFD3F0BD4FF6FF710160002195
:10075000017141718171C171704708B54FF48032E8
:100760000092009A0A430092009AC261C161009A05
:10077000C261C2690092C269009208BD02460020AF
:1007800013690B400BB1012000E0002070470146C7
:10079000086980B270470246002053690B400BB1D4
:1007A000012000E0002070470146486980B2704790
:1007B00001837047418370470AB1018300E04183A0
:1007C00070474161704742694A4042617047F0B5E5
:1007D000002300244D07ED0E02FA05F3CE1000F1C0
:1007E000200555F826504E07F70E0F26BE40B5439C
:1007F000CF1000F1200646F82750CE1000F120055A
:1008000055F8265045EA0304CE1000F1200545F8BE
:100810002640F0BD000002400004024000080240F3
:10082000000C024000100240001402400018024078
:10083000001C024000200240002402400028024028
:10084000F948006840F00100F74908600020F649C7
:1008500008310860F4480068F4490840F24908602B
:10086000F348091D0860F348EF4984310860F048F7
:100870001038091D0860EC48006820F48020EA491F
:1008800008600020E8490C310860E7498C310860B5
:1008900070470021E44A921C11701146087070479D
:1008A00010B501460022002300204A11012A02D17E
:1008B000DD4C236808E0022A03D1DB4C7034236846
:1008C00002E0D94C7434236801F01F0201249440E3
:1008D0001C400CB1012000E0002010BD38B5002004
:1008E00000900024002500BF3120FFF7D9FF054606
:1008F0000098401C00900098B0F5A04F01D0002D4A
:10090000F2D03120FFF7CCFF08B1012400E0002431
:10091000204638BD01460020C34A106820F0F80088
:1009200040EAC10010607047C34908607047002169
:10093000BD4A703211701170012802D004280AD10A
:1009400004E00121B84A7032117005E00521B64A71
:100950007032117000E000BF00BF7047B7490860F7
:10096000704770B5049C41EA82150126C6EB530618
:1009700045EA0645054345EA0465AB4E361D35603C
:1009800070BDAD4908667047820142EA0172A64B0C
:1009900084331A607047A8498866704710B5830190
:1009A00043EA016343EA02739F4C8834236010BD1D
:1009B000A14908677047A049C864704702460020F3
:1009C000994B0833186820F0EC6042EA01031843A1
:1009D000954B08331860704702460020924B08334D
:1009E000186820F0784042EA010318438E4B083320
:1009F00018607047014600208B4A0832106820F0CA
:100A0000030008431060704787480830006800F012
:100A10000C00704701460020834A0832106820F01D
:100A2000F000084310607047014600207E4A0832FB
:100A3000106820F4E0500843106070470146002021
:100A4000794A0832106820F4604040EAC100106022
:100A50007047F0B500210022002402250026022361
:100A6000714F08373F6807F00C0121B1042905D008
:100A7000082937D105E0724F076036E0714F0760F3
:100A800033E0694F3F1D3F68C7F38056664F3F1DF7
:100A90003F6807F03F036EB16A4FB7FBF3F7DFF82B
:100AA00088C10CF1040CDCF800C0CCF3881C07FBF7
:100AB0000CF40CE0624FB7FBF3F7DFF86CC10CF1FC
:100AC000040CDCF800C0CCF3881C07FB0CF4564F78
:100AD0003F1D3F68C7F301477F1C7D00B4FBF5F75E
:100AE000076002E0564F076000BF00BF4E4F083757
:100AF0003F6807F0F0010909534F7A5C0768D74057
:100B00004760494F08373F6807F4E051890A4E4F64
:100B10007A5C4768D7408760434F08373F6807F4DF
:100B20006041490B484F7A5C4768D740C760F0BDC9
:100B3000002100F44072B2F5407F0AD13A4A0832EF
:100B4000116821F4F811414A02401143364A083233
:100B50001160354A70321268C0F30B031A43324BEE
:100B600070331A607047354944390860704733491B
:100B700040390860704736490860704701460020D8
:100B8000294A8C32106820F01F004A1E1043264A62
:100B90008C321060704701460020234A8C32106866
:100BA00020F4F8504A1E40EA02201F4A8C3210609E
:100BB0007047014600201C4A8C32106820F4401017
:100BC00008431060704701460020174A8C321068B5
:100BD00020F4400008431060704701460020124A8C
:100BE0008C32106820F44030084310607047194977
:100BF0000860704739B10C4A3032126802430A4B20
:100C000030331A6006E0084A303212688243064BDD
:100C100030331A607047F9B1034A34321268024324
:100C2000014B34331A601CE000380240FFFFF6EA43
:100C3000103000240030002000004742800E474260
:100C40000024F40000127A0014000020FFFCFF0FC3
:100C50005C014742E01147428F4A126882438E4B43
:100C60001A60704739B18C4A121D126802438A4BD0
:100C70001B1D1A6006E0884A121D12688243864BCB
:100C80001B1D1A60704739B1834A0C321268024347
:100C9000814B0C331A6006E07F4A0C3212688243A3
:100CA0007D4B0C331A60704739B17B4A10321268A1
:100CB0000243794B10331A6006E0774A103212680B
:100CC0008243754B10331A60704739B1724A243A27
:100CD00012680243704B243B1A6006E06E4A243AC5
:100CE000126882436C4B243B1A60704739B16A4AE0
:100CF000203A12680243684B203B1A6006E0664ABD
:100D0000203A12688243644B203B1A60704739B125
:100D1000614A1C3A126802435F4B1C3B1A6006E0B2
:100D20005D4A1C3A126882435B4B1C3B1A60704759
:100D300039B1594A143A12680243574B143B1A60AE
:100D400006E0554A143A12688243534B143B1A602A
:100D5000704739B1504A103A126802434E4B103B6B
:100D60001A6006E04C4A103A126882434A4B103B24
:100D70001A60704739B1484A1C3212680243464B28
:100D80001C331A6006E0444A1C3212688243424B0C
:100D90001C331A60704739B13F4A2032126802434F
:100DA0003D4B20331A6006E03B4A203212688243F2
:100DB000394B20331A60704739B1374A24321268F0
:100DC0000243354B24331A6006E0334A243212685A
:100DD0008243314B24331A60704739B12E4A2C328A
:100DE000126802432C4B2C331A6006E02A4A2C323C
:100DF00012688243284B2C331A60704739B1264A57
:100E0000303212680243244B30331A6006E0224A23
:100E1000303212688243204B30331A607047012809
:100E200008D11D493C31096841F008011A4A3C3299
:100E3000116007E018493C31096821F00801164AA1
:100E40003C321160704739B1134A273A1278024395
:100E5000114B273B1A7006E00F4A273A127882435B
:100E60000D4B273B1A7070470B484030006840F02C
:100E70008070094940310860704701460020064AE9
:100E8000283A12680A400AB1012000E000207047A9
:100E900001492639087070473438024010B50446BD
:100EA000FA48844208D101211020FFF752FF0021A7
:100EB0001020FFF74EFF57E0F548844209D1012189
:100EC0004804FFF735FF00214FF40030FFF730FFF3
:100ED0004AE0F048844209D101218804FFF728FF45
:100EE00000214FF48020FFF723FF3DE0EA488442D1
:100EF00009D10121C804FFF71BFF00214FF4002096
:100F0000FFF716FF30E0E548844209D101210805CA
:100F1000FFF70EFF00214FF48010FFF709FF23E0D9
:100F2000DF48844208D101212020FFF712FF002171
:100F30002020FFF70EFF17E0DA48844209D1012193
:100F40008807FFF7F5FE00214FF08040FFF7F0FE25
:100F50000AE0D548844207D101214005FFF7E8FEA9
:100F600000216005FFF7E4FE10BD2DE9FF470546AF
:100F70000E460024A14600BFA046B08900B100BFC4
:100F80002C8A24F44054F08804432C82AC8941F22A
:100F90000C608443B0883189084371890843044355
:100FA000AC81AC8A24F44074B0890443AC826846B6
:100FB000FFF74FFDB548854202D0B948854202D1BE
:100FC000DDF80C9001E0DDF80890A88900F40040FD
:100FD00040B109EBC90000EB091031684900B0FBD2
:100FE000F1F707E009EBC90000EB0910316889004F
:100FF000B0FBF1F76420B7FBF0F004012009642195
:1010000001FB1078A88900F4004040B1322000EBC9
:10101000C800B0FBF1F000F00700044308E0322004
:1010200000EB08106421B0FBF1F000F00F00044366
:101030002C81BDE8FF874FF41651016000218180AB
:10104000C18001810C21418100218181704710B54F
:1010500002460020108A20F470600B884C882343DD
:101060008C882343CC8823431843108210BD002171
:10107000018041808180C180704721B1828942F422
:101080000052828104E082894DF6FF731A4082810A
:101090007047028B02F47F420283028B0A43028371
:1010A000704721B1828942F40042828103E0828943
:1010B000C2F30E028281704721B1828A42F400623B
:1010C000828204E0828A4FF2FF731A408282704764
:1010D000C1F308028280704701468888C0F3080087
:1010E0007047028A4FF6F0731A400282028A0A435E
:1010F0000282704721B1828942F00202828104E0BB
:1011000082894FF6FD731A408281704782894FF2BF
:10111000FF731A40828182890A4382817047028A62
:101120004FF6DF731A400282028A0A430282704736
:1011300021B1028A42F48042028204E0028A4BF624
:10114000FF731A4002827047818941F00101818159
:10115000704721B1828A42F00802828204E0828ACA
:101160004FF6F7731A4082827047028BD2B2028325
:10117000028B42EA01220283704721B1828A42F047
:101180002002828204E0828A4FF6DF731A40828254
:10119000704721B1828A42F01002828204E0828A82
:1011A0004FF6EF731A4082827047828A4FF6FB73C4
:1011B0001A408282828A0A438282704721B1828ADF
:1011C00042F00202828204E0828A4FF6FD731A40E6
:1011D000828270471AB1838A0B43838202E0838A3A
:1011E0008B4383827047F0B5034600240026002518
:1011F000002040F66A17B94200D100BF1846C1F37B
:10120000421401F01F06012707FA06F5012C01D14F
:101210000C3004E0022C01D1103000E014301AB17F
:1012200007682F43076002E00768AF430760F0BD1F
:1012300002460020B1F5007F00D100BF13880B40AB
:101240000BB1012000E00020704701F40072B2F5FC
:10125000007F00D100BFCA430280704770B50246CC
:10126000002400230025002040F66A16B14200D178
:1012700000BFC1F3421501F01F03012606FA03F374
:10128000012D13D19689334017E000000010014072
:101290000044004000480040004C00400050004026
:1012A0000014014000780040007C0040022D02D173
:1012B000168A334001E0968A33400C12012606FA62
:1012C00004F41688344013B10CB1012000E0002072
:1012D00070BD10B50022002340F66A14A14200D16F
:1012E00000BF0A1201249440A3B2DC43048010BD65
:1012F00010B504466FF00400FFF73AF9E11704EB6C
:101300005171C1F3C701394A11701046007800EBE2
:101310004001C1EBC0104FF6FF7101EAC000344933
:10132000088010BD0146314A12784A434FF0E0234D
:101330005A6100229A611A46126942F001021A614A
:1013400000BF4FF0E022106900F001021AB100F472
:101350008032002AF5D04FF0E022126922F001021B
:101360004FF0E0231A6100229A6170470146204A3B
:1013700012884A434FF0E0235A6100229A611A46CC
:10138000126942F001021A6100BF4FF0E0221069B9
:1013900000F001021AB100F48032002AF5D04FF0BB
:1013A000E022126922F001024FF0E0231A610022CC
:1013B0009A61704770B504464FF4077094FBF0F0E3
:1013C000C6B24FF4077094FBF0F100FB114085B2F8
:1013D00005E04FF40770FFF7C9FF701EC6B2002E7C
:1013E000F7D115B12846FFF7C1FF70BD24000020DA
:1013F0002600002000BF704700BF4C4A128802F050
:101400004002002AF9D0C2B2484B9A80704710B50A
:1014100088B0044601210846FFF7ECFB01211020AB
:10142000FFF742FC072209214148FFF7D0F90722C4
:101430000A213F48FFF7CBF94FF4C0600690022025
:101440008DF81C008DF81D0000208DF81E00012075
:101450008DF81F0006A93648FFF72EF902940020E8
:10146000ADF80C00ADF80E00ADF81000ADF81400AA
:101470000C20ADF8120002A92C48FFF776FD0121DF
:101480002A48FFF7FAFD012240F225512748FFF7CD
:10149000AAFE25208DF8040003208DF805008DF8A4
:1014A000060001208DF8070001A8FFF714F808B026
:1014B00010BD10B540F225511C48FFF7CFFE10B308
:1014C0001A48FFF709FEC4B21A48008800F4004029
:1014D000C8B91848008800F4804060B10A2C03D0D5
:1014E00000201449088020E01248008840F40040A1
:1014F0001049088019E00D2C06D10E48008840F4F0
:1015000080400C49088010E00A480088C0F30D00B4
:1015100009490C5407480088401C064908800846C1
:101520000088C72801DD0020088010BD00100140A0
:10153000000002402C000020300000207047000016
:101540000FB4044910B503AA029800F0D3F810BCF8
:101550005DF814FB280000202DE9F0410E460446FA
:10156000002020622046E168884730B3252805D056
:10157000D4E901219047206A401CF2E7E168204647
:1015800000278847050018D0A5F14100192802D886
:1015900020354FF400673246294620462760FEF783
:1015A0002DFE40B1012804D0F61D26F007060836AE
:1015B000D8E7361DD6E72846DAE7206ABDE8F0818D
:1015C0002DE9F0410646002410687529314616A51C
:1015D00010D0AFF30080002802DA404213A507E0E4
:1015E00031688A0701D512A502E0490704D511A583
:1015F000012401E0AFF3008000210A2206F1240754
:1016000009E0B0FBF2FCB0FBF2F302FB1C0030304F
:1016100078541846491C0028F3D123462A46304600
:10162000BDE8F04100F00CB8000000002D00000003
:101630002B00000020000000704770477047704783
:101640002DE9F0470D4699469246044600F12408DC
:101650000168880604D5E06921F01001216000E0EE
:101660000120A84201DD471B00E00027A1697A198B
:1016700002EB0900081AA0612078C00602D42046B7
:10168000AFF30080002608E0D4E901211AF8060033
:101690009047206A401C761C20624E45F4DB20787F
:1016A000C0060AD52046AFF3008006E0D4E9012148
:1016B00030209047206A401C2062381EA7F10107A5
:1016C000F4DC07E0D4E9012118F805009047206A0E
:1016D000401C2062281EA5F10105F3DC2046AFF373
:1016E00000802078000602D50220BDE8F0870120A6
:1016F000FBE70000074B70B50D467B4400F011F886
:101700000446284600F020F810B14FF0FF3070BDBD
:10171000204670BDFBFCFFFF01694A1C026108788E
:10172000704700B58FB0CDE9013100210591054921
:101730007944CDE9031011466846FFF70DFF0FB05D
:1017400000BD0000E5FFFFFF007B00F08000704758
:10175000754600F02BF8AE4605006946534620F06A
:101760000700854618B020B5FEF79EFEBDE8204074
:101770004FF000064FF000074FF000084FF0000B4D
:1017800021F00701AC46ACE8C009ACE8C009ACE800
:10179000C009ACE8C0098D46704710B50446AFF3E8
:1017A00000802046BDE81040FEF73CBD0048704771
:1017B000F80000204FF04070E1EE100A7047000082
:1017C000E01700080000002030000000C4010008FD
:1017D000101800083000002028070000E001000871
:1017E000007A030A00000000000000000102030468
:1017F00006070809000000000102030401020304B7
:1018000006070809000000000000000000000000BA
:040000050800018965
:00000001FF
